:020000040000FA
:10000000C0070020D5000000DD000000DF00000078
:1000100000000000000000000000000000000000E0
:10002000000000000000000000000000E1000000EF
:100030000000000000000000E3000000E9210000D3
:10004000000000000000000000000000E7000000C9
:10005000E7000000FD0800003909000075090000F4
:100060000000000000000000000000000000000090
:100070006D08000031220000E7000000512200005E
:100080000000000000000000000000000000000070
:10009000C90A0000E700000000000000E7000000BF
:1000A0000000000071220000C922000000000000D2
:1000B0000000000000000000000000000000000040
:1000C0000348854600F010FB00480047E534000077
:1000D000C00700200448804704480047FEE7FEE7C9
:1000E000FEE7FEE7FEE7FEE711220000C100000088
:1000F00030B50B46014600202022012409E00D46C0
:10010000D5409D4205D31D469540491B2546954047
:1001100040191546521E002DF1DC30BD03460B433D
:100120009B0703D009E008C9121F08C0042AFAD2AD
:1001300003E00B780370401C491C521EF9D2704733
:10014000D2B201E00270401C491EFBD2704700226F
:10015000F6E710B513460A4604461946FFF7F0FFC6
:10016000204610BD0321001D401E037812021A43D1
:10017000491EF9D510467047034603220870000A4D
:10018000491C521EFAD518467047024670B54A40BF
:10019000D30FDB0740002DD04A002AD0010E140EE9
:1001A000000212020919400A520A8418E5010446A5
:1001B0005443000A120A2E045043A4194219200C79
:1001C000C543AA18120C0125AD03521C5219120482
:1001D0007F39240400D0521C104301D44000491E32
:1001E000C2B20C06C0092018401C4008802A02D068
:1001F00003E0002070BD40084000002900DA002024
:10020000184370BD420005D04200120E52428A428D
:1002100001DB00207047C9050818704710B500229F
:100220009623114600F061F810BD41004002012202
:10023000400AD205090E80187F2901DA0020704794
:10024000962903DC9622511AC84070479639884097
:100250007047C20FD207400040080BD0C10D0723E2
:10026000DB01C91840020905400A1143C2084007D2
:1002700011437047002001467047F0B51FB4064691
:10028000002082B005464024019100901BE00199B6
:1002900022460F46304600F049FA049A059B801A20
:1002A000994110D310461946224600F02FFA361A0B
:1002B0008F410197224601200021009F00F026FA7D
:1002C00038184D4100902046641E0028DFDC019B59
:1002D00000982946324607B0F0BD002904DA401CD8
:1002E000490001D140084000704770B40024050C5B
:1002F00005D11024000402D1002921D01124050EBB
:1003000001D100020834050F01D10001241D850F21
:1003100001D18000A41C002801DB4000641C0029DE
:1003200008D020252E1B0D46F540A14000D001210C
:100330002943084301061B1B000ADB1D02D50020D0
:1003400070BC7047DB05181880180029F8DA401CCB
:100350004900F5D170BC400840007047F0B5074631
:100360000846584087B0C00F049048000E46590018
:1003700040084908BC1A884105D2384631461E4615
:1003800017460B4602465800400810434CD0300D2B
:10039000039040055900400D490D0590401A029008
:1003A000402872DA18030121000B09050843019067
:1003B00004980092002805D00199524200208841FB
:1003C00000920190029840210A1A0199009800F0C9
:1003D0009DF905460C466B4607CB00F0B8F9C019ED
:1003E0007141039A0E0D0023D71756401A467A40E2
:1003F000164344D0049A002A2DD0029A012A039A67
:1004000015DC1205C01A914101263605001C714108
:10041000D20F059ED2070093019202962A462346E8
:1004200000F0B5F907B0F0BD38463146FAE71605D9
:10043000224A0F46B218C01AB74101210905001C13
:100440004F4100187F41114618187941E20F1043BF
:100450006D19644113E0E2076D0815436408C20793
:100460001443039A01261205C01A91413605001C57
:100470007141CE07400830434908C01851412A460F
:10048000234600F077F9CDE7FFE70498012240000A
:10049000C117121A00238B4104983146C417381A29
:1004A000A141EEE730B40124E407634030BC55E7D6
:1004B00030B40124E407614030BC4FE70000E0FFA6
:1004C000F0B51FB488B00B990998002448400999E9
:1004D000C00F490049080991C0070B9900904900D5
:1004E00049080B9109990898A64608431CD00B9916
:1004F0000A98084318D0099801244000420D48008A
:10050000410D099824050003000B204309900B9826
:100510000003000B20430B9050181C494018002288
:1005200001901446104605E0002001460DB0F0BDD4
:10053000032801DA034600E003239C46C11A0AAEF1
:100540000AE05F0008ADED5B4F00F75B7D430027DD
:10055000AA187C41491C5B1E6145F2DD410004ABD9
:100560005A522104120C0A43240C401C0828DFDBD9
:10057000019802900099704601910090059B049AA1
:100580000799069800F003F9D0E700000DFCFFFF83
:10059000F0B50C465C4085B0E40FE40703944C00D2
:1005A00000266408590094464908024602962243F0
:1005B00021D062460A431ED06200570D4A000E0346
:1005C0002303550D012402462C492405781B1B0BDF
:1005D000360B401823432643614600901C46501AB0
:1005E000B44103D30098401C009002E09218009898
:1005F0005B41002803DA0020014605B0F0BD002071
:10060000012109050746864611E064461D46141B74
:10061000B54106D36546521BB341744607430C43AC
:10062000A646CD0740084908284392185B41054675
:100630000D43EAD11046184313D060461946504086
:100640007140084306D06046101AB34106D2012219
:10065000002306E000220123DB0702E00122D2434F
:100660005310009874460105381C6141029C039D9B
:100670000019694100F07EF8BFE70000FD030000AB
:100680004A0009030123090B1B0519430A4B10B546
:10069000520D9A4202DA0020014610BD064B343357
:1006A0009A4203DC9A1A00F041F810BD034BD218AD
:1006B00000F02CF810BD0000FF030000CDFBFFFF91
:1006C00010B5002904DB0124E40740428C41214697
:1006D000002B04DB1C460123DB075242A341994255
:1006E00000D1904210BD0000064C0125064E05E0E9
:1006F000E36807CC2B430C3C98471034B442F7D343
:10070000FFF7E2FC245200004452000010B5202AFA
:1007100004DB0146203A9140002010BD9140202387
:100720009C1A0346E3401943904010BD10B5202A9F
:1007300004DB0846203AD040002110BD0B46D340D0
:10074000D0402024A21A91400843194610BD10B58C
:10075000202A06DBCB170846203A1041C1170B436D
:1007600006E00B461341D0402024A21A91400843D2
:10077000194610BD10B5002B08DA0024401C614159
:1007800092185B411A4301D14008400010BDF0B5FA
:100790001FB482B005460C0003D0084601F0D0FD1E
:1007A00002E001F0CDFD20300246009021462846AF
:1007B000FFF7ACFF049B059A04460F46184311430C
:1007C000084314D0184610431BD0009840210A1A41
:1007D00018460599FFF7AAFF05460E46009A0599A7
:1007E0000498FFF793FF084305D0012004E020465A
:1007F000394607B0F0BD0020C11705430E432C4316
:10080000374300990E986305401A7905E40A0022DF
:100810000C43FD0A0A3002D500200146E9E7010534
:10082000101969410C9C0D9D00196941FFF7A2FF49
:10083000DFE730B58C180278401C13071B0F01D17D
:100840000378401C120906D10278401C03E00578A9
:100850000D70401C491C5B1EF9D101E00B70491C56
:10086000521EFBD1A142E6D3002030BD70B504205A
:1008700003F0C4FE104E114C114D002809D0042085
:1008800030610D4840300168A0784200A952401CF8
:10089000A070082003F0B2FE00280BD008203061C1
:1008A000A078400040194038C08F03F099FE606086
:1008B0000020A07070BD00000024014060000020F6
:1008C000FC03002010B504490120486002460221C3
:1008D000024801F041F910BD003001400004005011
:1008E00010B504490020486002460221024801F088
:1008F00033F910BD003001400004005070B50325ED
:100900006D06284603F0CCFE094C002804D028468A
:1009100003F0B0FE20688047064D284603F0C0FE75
:10092000002804D0284603F0A5FE6068804770BD0B
:10093000A00000200100000670B50C4D284603F011
:10094000AFFE0B4C002804D0284603F093FEA068AD
:100950008047064D6D1C284603F0A2FE002804D0F7
:10096000284603F087FEE068804770BD020000065D
:10097000A000002070B5184D284603F091FE174CDA
:10098000002804D0284603F075FE20698047124DE8
:100990006D1C284603F084FE002804D0284603F08E
:1009A00069FE606980470C4DAD1C284603F078FE57
:1009B000002804D0284603F05DFEA0698047064D5C
:1009C000ED1C284603F06CFE002804D0284603F0F6
:1009D00051FEE069804770BD04000006A0000020C1
:1009E00004484178002903D101214170322141613D
:1009F00070470000E003002010B5054CA1780029E5
:100A000005D10121A1700A21FFF772FBE06010BD42
:100A1000E00300200149012008707047E003002036
:100A200070B52749002648764A69002A02D0521E2E
:100A30004A6100E04E70224A224B147A01220028BB
:100A40002AD0CD68002D01D06D1ECD600D7EA8424C
:100A500013D18D78002D07D0CD68002D04D18D796C
:100A6000002D00D11A708A71CD78002D0DD0CD687F
:100A7000002D0AD11A70CA7107E04D78002D04D0FC
:100A80004D69002D01D01A704A71002C00D11A70E6
:100A900008760E710A720EE00D78002D04D0002C3D
:100AA00003D01A700A7100E00876CE708E708E71D5
:100AB000CE714E710E72087E5870024870BD0000F3
:100AC000E00300205C000020FEB504F0A1F84249DC
:100AD00002220868104002287DD148603FA001F042
:100AE0001FFC434CA07E411CA176002873D0002639
:100AF000A67602F09FFB207B1F277F013D4D00283B
:100B000007D0607B002866D13B486062012060739B
:100B100023E0607A00285ED0A06A00285BD0401EE7
:100B2000A06258D135486062A07B002812D0B42062
:100B3000A062207902280AD3267160791128A07951
:100B400002D002F099F908E003F032F905E0401C08
:100B5000207102E0E1208000A062694648784009E7
:100B60004001153048708878497800020843A97818
:100B7000B843C906890D084369464870000A887061
:100B8000C0B2F3210840E97A8907090F0843694692
:100B90008870E81DFFF7E6FA02016946488809797E
:100BA0000904084316490840024369464A80100C6C
:100BB000087102F03FFB01A90131FFF7DDFA0146A0
:100BC00010A001F0ADFB0A21684602F0C1F90A212C
:100BD000684603F0F9FBFEBD007C00404C505449D0
:100BE0004D315F49525148616E646C65720D0A0067
:100BF0000000002030010020204E0000881300007B
:100C00000F0000FF6261744C6F77566C7453656E11
:100C100064466C6167202025640A000010B5042139
:100C2000024800F047FFC0B210BD000000040050B1
:100C3000F8B50020009008223E21022000F05AFA68
:100C40001B4E00246D4620461E30C2B231463B206A
:100C500000F0F4F92855641C032CF4D31C2231460F
:100C60003B2000F0EBF95A281BD1FD223D21022048
:100C700000F0E5FC68468278002A03D04521002078
:100C800000F0DDFC684600781C21C206D20E03206D
:100C9000C03200F0D4FC684642781D21032000F0E9
:100CA000CEFC08223E21022000F04AFB0020F8BDC5
:100CB000A55A000010B502466C21002000F0BFFCD0
:100CC00010BD000010B501220621022000F012FA2A
:100CD0002823064A0A21022000F0D5FCEF22342105
:100CE000022000F0ACFC002010BD00001C510000F0
:100CF00070B5074D00246000201841198A784978A2
:100D0000285C00F09CFC641C392CF4D3002070BDDE
:100D1000F14E000010B50122134683400446083C02
:100D2000A240002903D0012909D0012010BD0828C4
:100D300002D2DAB2632109E0D2B2642106E00828C7
:100D400002D2DAB2652101E0D2B26621002000F0C1
:100D5000F7FA002010BD000010B5162000F064FB6B
:100D60000F4800F04FFA072000F0D4F9092000F0F6
:100D700039FB012000F0E8F9012000F0F3F9002030
:100D800000F0C2FAAA2000F0EBFA002000F0A4FA6A
:100D9000002000F0F7FA002000F0F2F910BD00008A
:100DA000400ECF1910B504467D21C90061430846A5
:100DB00000F001F810BD10B50446204603F03CFCDD
:100DC00010BD10B5042000F0EDFA00F0F7FB00F0C4
:100DD000D5FB022000F0F2FA062000F0E3FA10BD85
:100DE00010B50446042000F0DDFA00F0E7FB00F047
:100DF000C5FB204600F0EAFA012000F0DFFA0620E9
:100E000000F0D0FA10BD000010B500F06FFB042117
:100E1000022000F044FC9620FFF7CDFF03210220C2
:100E200000F03DFC0A20FFF7C6FF0221084600F053
:100E300036FC0A20FFF7BFFF1621042000F02FFC2C
:100E40000A20FFF7B8FF0121022000F028FC0A2049
:100E5000FFF7B1FF20220621032000F04BF90A2002
:100E6000FFF7A9FF00222621032000F0E8FB02493A
:100E70000120C87010BD00002801002010B504201A
:100E800000F090FA01490420C87010BD280100202C
:100E900010B520220621032000F052FA0A20FFF7A5
:100EA0008AFF0221084600F0FAFB0A20FFF783FFC1
:100EB00020222621032000F0C2FB6420FFF77BFFE5
:100EC0003621042000F0EBFB6420FFF774FF0321C0
:100ED000022000F0E4FB0120FFF764FF0421022060
:100EE00000F0DDFB6420FFF766FF02490420C870B4
:100EF00010BD00002801002010B56C21002000F07A
:100F0000BFF84006400E10BD0148C0787047000091
:100F10002801002010B57F21012000F0B1F840B277
:100F200010BD70B5054600F008F804460246294693
:100F3000012000F0BCF8204670BD10B57D210120D5
:100F400000F09EF810BD000010B5FFF767FE002806
:100F500003D0024901200968884710BD2401002000
:100F600010B50621042000F09AFB6420FFF723FF50
:100F70000321002000F093FB03211A2000F08FFBD7
:100F8000002000F0CFF90021022000F088FB0A20A9
:100F9000FFF711FF0121022000F081FB0A20FFF77B
:100FA0000AFF20220621032000F049FB0A20FFF758
:100FB00002FF0221084600F072FB0A20FFF7FBFE49
:100FC00020222621032000F03AFB6420FFF7F3FEE5
:100FD0003621042000F063FB0120FFF7E3FE03212C
:100FE000022000F05CFB0120FFF7DCFE0421022060
:100FF00000F055FB6420FFF7DEFEFFF779FEFFF7F8
:1010000017FEFFF75FFE00F007F802490420C870E2
:10101000002010BD2801002010B501210A20FFF793
:1010200079FE01210020FFF775FE00210A2000F063
:10103000F3FA0021084600F0EFFA10BD38B5054676
:101040000B0A684603704170510081700B4C0323FA
:101050006A462946022000F016FB6C21002000F0B1
:101060000FF8000604D42046641EA4B20028F4D170
:101070002946022000F004F838BD000010270000C7
:1010800010B50C4600F04EF9204600F001F810BDF6
:1010900010B50446FFF724FC6006000E02F0C0FE07
:1010A00001F09CF80446FFF70DFC204610BD70B51A
:1010B00015460E460446FFF713FC6006000E02F0CC
:1010C000AFFE002404E001F089F83055641CE4B25E
:1010D000AC42F8D3FFF7F6FB70BD10B580210020BD
:1010E00000F0DDFA0021084600F0D9FA0020FFF7F1
:1010F000CFFF10BD70B514460D4600F013F9284619
:10110000FFF7C6FFA0430146284600F0C8FA0020BA
:1011100070BD000010B504460246F0230D210320E7
:1011200000F098FA092C05D002223F21104600F069
:1011300007F904E002223F211046FFF7DBFF0148D8
:10114000447210BDA805002010B5044602460E23C7
:101150000D21032000F07EFA0148847210BD0000CA
:10116000A805002010B50446024608230E210320DE
:1011700000F070FA0148C47210BD0000A8050020FC
:1011800010B5040020D0F02304222521012000F016
:1011900061FA012208232521104600F05BFA04239E
:1011A00000221221032000F055FA10230022122100
:1011B000032000F04FFA042300225821002000F001
:1011C00049FA0F48847410BDF02300222521012024
:1011D00000F040FA082300222521012000F03AFA0D
:1011E000042301221221032000F034FA10230122EB
:1011F0001221032000F02EFA04230122DDE7000073
:10120000A8050020FEB50446002002902C482027A7
:1012100084422AD32B48806FA04226D32A48002537
:101220000C2169434258A2421AD209184968A142C6
:1012300016D30C2169430E18B07A23494006400F9B
:10124000F839085C3246604302900832022340219C
:10125000002000F018FAB17A3D2000F020FA02E0F8
:101260006D1CBD42DCD3BD4201D30120FEBD174938
:101270000298FEF73DFF06460846143E1449FEF765
:1012800037FF054669460C70200A4870200C8870AC
:10129000200EC87004236A460921032000F0F3F9E8
:1012A00069460E7128054D71000F8871032301AA4C
:1012B0001521184600F0E7F9064844600020FEBDFD
:1012C00090BF3E089C5000009C4F00000048E80181
:1012D000409C0000A805002010B50A4C002807D04B
:1012E000012260230E21104600F0B4F9012006E02F
:1012F000602302220E21012000F0ACF900202073AF
:1013000010BD0000A805002010B5044602460823C1
:101310001221032000F09EF90148847310BD0000E3
:10132000A805002010B505490A78824204D008704B
:101330000146002000F0B3F9002010BD2801002074
:1013400070B515460C46FFF7EDFF2046FFF7A0FEEF
:1013500028430146204600F0A2F9002070BD00009D
:1013600038B5044668460470210A417002236A4673
:101370001321032000F087F90148048238BD0000E2
:10138000A805002010B50446012807D0002224211A
:10139000032000F054F90248C47410BD0822F6E797
:1013A000A805002010B504460146022000F077F998
:1013B0000148C47010BD00002801002010B50323AF
:1013C00002460621184600F045F910BD08B56946E9
:1013D0000870000A487002236A460721032000F0C3
:1013E00052F908BD10B504460246F0230E21032031
:1013F00000F030F90148047210BD0000A80500207B
:1014000010B5044602460F21032000F018F90148E8
:10141000447310BDA805002010B502460423062120
:10142000032000F017F910BDF8B5162801D91620D1
:1014300002E0002800D101200646451E6800274C26
:101440002F183D1968782221C207D20F032000F01F
:10145000F6F8E25D1E21002000F0F1F868784B21DB
:101460000209002000F0EBF8A878702805D00422CB
:1014700046210020FFF764FF04E0042246210020FB
:10148000FFF738FE164C6078002816D101206070F6
:1014900008223E210220FFF72DFE202211493B2089
:1014A000FFF7CCFDA07008223E210220FFF748FF85
:1014B000A078002801D10820A070A978A278080798
:1014C000000F101A0A09C0B2120102434521002080
:1014D00000F0B5F804480670F8BD0000AC4E0000FE
:1014E00028010020A55A0000A805002010B5002101
:1014F0000A2000F091F80021084600F08DF810BD98
:1015000010B50421022000F0CAF80022582110462C
:1015100000F095F80120FFF77FFF01220C21104613
:1015200000F08DF800F038F80521022000F0B7F83F
:10153000FF21012000F0B3F801490520C87010BD5B
:101540002801002010B540225E210020FFF7F8FEA0
:101550000A220F21012000F072F8F4223521012027
:1015600000F06DF80420FFF71DFFFFF7B6FD0249FC
:101570000420C87010BD00002801002010B508220A
:101580004F210020FFF7B6FD10BD10B508224F21F6
:101590000020FFF7D5FE10BD10B50748C07C01281C
:1015A00004D100222421032000F049F8FFF7EDFFC9
:1015B00000F00EF810BD0000A805002010B50021B5
:1015C000084600F029F801210A2000F025F810BD96
:1015D00010B500210A2000F01FF80121002000F0C2
:1015E0001BF810BD70B50C4605460421022000F022
:1015F00056F80020FFF710FF22460C21012000F0D2
:101600001EF8FFF7C9FF0520FFF7CCFE224629464A
:10161000012000F055F870BD10B50123082804D250
:1016200083400A46DBB2672104E0083883400A465B
:10163000DBB26821002000F00DF8002010BD70B56D
:1016400014460D46FFF76EFE2146284600F027F8A7
:10165000002070BD70B51D46034614460E46284650
:1016600000F0C0FE8440E4B22C401846FFF75AFE5A
:101670003046FFF70DFDA84320430146304600F0F9
:101680000EF8002070BD70B51C4615460E46FFF7DB
:1016900049FE22462946304600F012F870BD70B56A
:1016A0000C460546FFF71CF96800401CC0B202F06A
:1016B000B7FB204602F0B4FBFFF704F9002070BD31
:1016C00070B515460E460446FFF70AF96000401C47
:1016D000C0B202F0A5FB002404E0305D02F0A0FBE4
:1016E000641CE4B2AC42F8D3FFF7ECF870BD000024
:1016F00001494000085A7047FC030020F0B585B04E
:10170000054602F081FF2F4614216846FEF71FFDB3
:10171000E806000F02D0012003F056F9E12005424F
:1017200002D0022003F050F903203C4E0024019027
:10173000F80713D0002C6AD0052C68D0062C66D090
:10174000072C64D036486100405A00900520694655
:10175000000703F088F87078401C70707F08641CE4
:10176000082CE5DB2F480122816B120511438163B0
:1017700000BF00BF00BF01212B4C4906A068072213
:10178000120690430843A060606803214902884321
:1017900060606068A11403221203904308436060F4
:1017A000A1690720090909010143A16160680421B9
:1017B00088436060284689010843E1690143E1618B
:1017C000A068012109040843A060162002F034FF3C
:1017D0006068012189030843606014490868022297
:1017E0009043104308600120206002F025FF60054F
:1017F0002060070D384602F001FF0028FAD00C489F
:101800002061307828433070E8B205B0F0BD04485C
:101810006100405A0090694606489AE7600000203F
:10182000D84D000000100240002401400026014075
:101830009E0800000004005010B502484068FEF702
:10184000EDFC10BD60000020F8B5134D04202860A9
:10185000114F0024114E40370BE0042002F0CEFE61
:101860000028FAD0386861007052641C0420E4B289
:101870002861082002F0C2FE0028EED0082028616E
:1018800010202860600080194038C08F02F0A8FE48
:1018900003494860F8BD000000240140FC0300201B
:1018A00060000020FFB589B00E4607461C460025A3
:1018B000142104A8FEF74BFC002000900190029038
:1018C000039005200007874204D1012003F0A4F80B
:1018D00000200EE03148874204D1022003F09CF83A
:1018E000012006E02E48874204D1042003F094F83A
:1018F00002200390002005900B980690049604A9FE
:10190000384602F0B0FF00206D1CEDB2F10703D1A4
:101910007608401C0828F7DB6E1E2248330000F0D2
:1019200026FD080507090B0D0F11131404600CE0C8
:1019300044600AE0846008E0C46006E0046104E0FA
:10194000446102E0846100E0C4611749A8004018C6
:101950008038C06F00900120019012980290684674
:1019600002F0A8FE012E05DC0520139900F018FDF9
:1019700005200EE0032E05DC0620139900F010FD73
:10198000062006E0072E06DC0720139900F008FD6C
:10199000072000F0F9FCF0B20DB0F0BD00040050DB
:1019A00000080050A00000206C4E000010B500237D
:1019B00003E0C45CCC545B1C9BB29342F9D310BDD2
:1019C000FEB50C4696089107890F0291154600272F
:1019D0003449334A01970A614969002904DA3149D7
:1019E000314A8A60314A8A604002014600900420F0
:1019F00002F0E0FE00283DD1002E1CD0019815E039
:101A0000019900208A001118615CC30099400F43BE
:101A1000401C0428F7DB00983946801802F0FAFED3
:101A2000002827D101980027401C0190B042E7D33D
:101A3000029800281FD00298012804D0022808D05C
:101A4000032825D118E060192038C17FFF20C0434A
:101A500006E060192038C17F0A02817F14481143D3
:101A600001430098002E01D0B200801802F0D2FE8F
:101A700000280FD00120FEBD60192038C17F827F71
:101A8000090412020A43417FFF2011430006E7E7E1
:101A90000020FEBD03484169820411434161F7E71C
:101AA0001000000100200240851A7AE591836E7CC7
:101AB0000000FFFF70B50C46054602F0CBFE002883
:101AC00001D0FF2070BD2869844301D0002070BD83
:101AD000012070BDF0B585B00F4605461E46144680
:101AE00014216846FEF733FB0522120711491248FC
:101AF000954201D1012002E08D4203D1022002F083
:101B000059FF03E0854201D10420F8E700970194D2
:101B1000002C04D000200290012C02D003E0029699
:101B200001E00A9803906946284602F09CFE05B041
:101B3000F0BD0000000400500008005070B50D46D4
:101B4000044602F087FE012801D0FF2070BD6069C5
:101B500068406061012070BD70B516460C460546B0
:101B600002F078FE012801D0012070BD012E02D0C4
:101B7000AC62002070BDAC61FBE70000F0B595B031
:101B8000044607460026142101A8FEF7E0FAA00645
:101B900002D0012002F022FFE005C00E02D0022098
:101BA00002F01CFF02200290002003900320002579
:101BB0000590F8071BD0062D07D23A486900405A15
:101BC0000190052001A900070FE0E81F022806D2B6
:101BD00034486900405A019001A9334805E0314872
:101BE0006900405A019001A9304802F03CFE6D1C8A
:101BF0007F08EDB20A2DDCD314210FA8FEF7A7FA57
:101C0000202106A8FEF7A3FA294902204A6B0243C5
:101C10004A6300BF00BF00BF08200F90B82011909A
:101C200001204002234D12900FA9284602F020FF08
:101C30002868E913084328601020069002200A90C3
:101C4000119801274008099049200797044205D0C0
:101C5000002206A9284602F035FF3E432420044214
:101C600006D0012206A9284602F02CFF02200643D6
:101C7000FF201330044206D0022206A9284602F0B3
:101C800021FF04200643200606D5032206A9284684
:101C900002F018FF082006432868384328603046C1
:101CA00015B0F0BDE84D00000004005000080050E1
:101CB000001002400004004070B586B004461421B4
:101CC0006846FEF744FA092C01D2012104E0112CE8
:101CD00001D2022100E00421092C02D205200007D4
:101CE00004E0112C01D2154800E01548154E0125DD
:101CF0007060092C02D22846641E05E0112C28468B
:101D000001D2093C00E0113CA0407080084602F07E
:101D100079FE70880090002001950290039069463A
:101D2000706802F0A0FD71687088886105480649F6
:101D3000083001600549416006B070BD00040050E4
:101D40000008005090000020E11E0000F11E00007D
:101D5000FFB589B00546142102A8FEF7F8F9002066
:101D600005273F07384C0190012D05D08026032D13
:101D700004D03D46012003E00126FAE72546022073
:101D800002F040FE0220039000200490059006908F
:101D9000029602A9284602F066FD0A98022837D06A
:101DA00001283BD00225294E042002F02BFE019889
:101DB0000690029502A9304602F055FD0B980128C5
:101DC00030D0002001900B98022831D004252646FF
:101DD000022002F017FE012004900198069002955F
:101DE00002A9304602F03FFD0C98012828D00026B9
:101DF00002281FD0032821D02025022002F002FE55
:101E000002A920460696029502F02DFD0DB0F0BD08
:101E100004204025019026460220C6E702253E46C2
:101E20000120C2E70420402501903E460120D0E772
:101E30000125CCE740253C460120DFE70225DCE711
:101E4000034901200870E1E7000400500008005039
:101E500090000020F7B586B00D46074600261421F5
:101E60006846FEF774F91B480122816B1203114387
:101E7000816300BF00BF00BF174C206840084000CE
:101E80002060402001970090002D11D0012D02D03C
:101E90002026022D0CD01020039008980490029662
:101EA000684602F0CDFD0D480078002802D00BE016
:101EB0000020F1E7206801218902084320600749DA
:101EC0000020083108604860206801210843206034
:101ED00009B0F0BD00100240003001409000002029
:101EE00002494868498881617047000090000020DD
:101EF00002494868498881627047000090000020CC
:101F000070B52C4E2C4C0546022805D0002002F05E
:101F10006DFC032D03D138E0012002F067FC20683E
:101F2000FF2101310843206088002168014081427F
:101F3000FBD1002D04D0012D0BD0022D1CD011E0BF
:101F4000002002F073FD02F011FD0028FBD11B48B8
:101F500007E0012002F06AFD02F008FD0828FBD12D
:101F600017483060A068072109028843A060A06874
:101F700009018843A06070BD022002F057FD02F005
:101F8000F5FC1028FBD10F48EBE70B4840304168C7
:101F90000122114341600222416811400229FBD114
:101FA000032002F043FD02F0E1FC1828FBD17D2064
:101FB0000002D6E7C00000200010024000127A00A4
:101FC0000024F400006CDC02FFB585B00F46054626
:101FD0001E4614216846FEF7BAF81F480122816B9D
:101FE000D2021143816300BF00BF00BF0020FF2168
:101FF000013103910090029501906946174C0874D5
:10200000204602F035FD0120C043206108202168F0
:10201000012F1FD08022114321602168814321605C
:102020000F4A1168FF231B029943B3071B0E0120BF
:102030001B02194311600B4A410311600A4A0799B8
:102040001160E1680143E160216801432160E8B269
:1020500009B0F0BD0143E2E700100240002C01404E
:102060000CE400E000E100E068000020FFB58DB066
:1020700007461C461546002614216846FEF767F8F9
:1020800002200190012002900020A10003900B91FA
:102090004D48A9000A91874246D1072C14D2032C3F
:1020A00005D2012002F0A4FC052636070CE0062C20
:1020B00004D2022002F09CFC444E05E0062C03D121
:1020C000042002F095FC424E424C0B986946205881
:1020D000009001200490304602F0C5FB0020072D3F
:1020E00011D90A2D09D2012002F082FC0520000737
:1020F000092D08D10521049105E00C2D03D2022001
:1021000002F076FC31480A9961580091694602F064
:10211000AAFB142105A8FEF71AF82F480121826BAB
:1021200089030A4382633AE0052004900F2C0DD204
:102130000E2C05D2012002F05BFC0526360705E0D7
:102140000E2C03D1022002F053FC204E214C0B98A0
:10215000694620580090304602F085FB00200E2D85
:102160000DD9112D05D2012002F042FC05200007F7
:1021700005E0112D03D1022002F03AFC13480A9920
:1021800061580091694602F06EFB142105A8FDF725
:10219000DEFF11480121426B49040A43426300BF3C
:1021A00000BF00BF0E9806900C20059000200790FD
:1021B0000890099005A9384602F008FD3868012109
:1021C0000843386011B0F0BD0038014000040050F1
:1021D00000080050244E00000010024010B5FF20FF
:1021E00001F01EFE10BD00000849087800280CD040
:1021F000002007E08200521853681A89521E401CC2
:102200001A81C0B20A788242F4D8704710040020C4
:102210000449034888600549034808607047000086
:102220000000000000ED00E000127A00C000002075
:1022300005480169C907C90F05D00121C9430161DA
:102240000248006800477047002C014068000020E9
:1022500005480169C907C90F05D00121C9430161BA
:102260000248006800477047000400406C000020EE
:1022700070B5134C20202168124D014217D0E0693F
:102280002021084213D0202020626878002802D044
:10229000E86880470BE0616AA888AA681154401C6E
:1022A00080B2A8802978884201D30020A880E16903
:1022B0000820014202D020622869804770BD0000DA
:1022C000003801407000002070B5134C20202168B8
:1022D000124D014217D0E0692021084213D020207E
:1022E0002062E878002802D0A86980470BE0616A84
:1022F000E888AA681154401C80B2E880A978884216
:1023000001D30020E880E1690820014202D0206268
:10231000E869804770BD0000004400407000002064
:102320000FB410B503A9044B044A029800F030F929
:1023300010BC08BC04B01847213200002C0100205A
:102340002021020C01D010211046020A01D01046B3
:102350000839020901D01046091F820801D0104631
:10236000891E420801D0881E7047081A704730B491
:102370007446641E2578641CAB4200D21D46635D22
:102380005B00E31830BC1847002805DBC106C90E06
:1023900001208840014908607047000000E100E02A
:1023A0008307FF22DB0E9A408907090E9940002817
:1023B00008DB830809489B001B18186890430843F2
:1023C000186070470007000F0838830804489B0016
:1023D0001B18D86990430843D861704700E400E0B7
:1023E00000ED00E000210246CA40D20701D0C8B289
:1023F0007047491C0829F6DB0020704702E008C836
:10240000121F08C1002AFAD170477047002001E06E
:1024100001C1121F002AFBD170470000F0B51FB4A4
:1024200086B00998089A030D0021024314D0514840
:10243000514A1818504305141198012810981AD0C1
:10244000281A401C00264D4F4D49009601910490DA
:10245000002812DA444211E01198012449A301280E
:1024600001D11098C1430698119A84600360C2603C
:1024700041600BB0F0BD4042E4E704462105002076
:102480003F4A001C51410391029012E0E00707D03F
:1024900032463B4601990098FEF712F801910090F0
:1024A00032463B4610461946FEF70AF806460F46E6
:1024B0006410002CEAD10498039B0028029A099921
:1024C000089806DAFDF7FCFF019B009AFDF7F8FF7C
:1024D00005E0FEF75DF8019B009AFEF759F8044607
:1024E0000E460022284BFEF7EBF803D80020C0432D
:1024F000014607E00022254B20463146FDF72EFF1E
:10250000FEF7BEF8102409E0002C0ADB0A220023A3
:10251000FDF7B3FE079B30321A55641E02460A438C
:10252000F2D11122641C079B121B1C19119B012B59
:1025300003D0012308430ED10AE0084304D0112040
:1025400010900020119077E71098151A6D1E0BE07F
:102550001098824202DD00236D1C03E0824201DA02
:1025600000236D1E002BEED0069811998260C16089
:1025700030C07EE701FCFFFF104D0000000014405A
:102580000000F03F300000000000F0430000E03F9A
:10259000FFB597B00646002518E2252877D100241C
:1025A0002746FD49049400E00443761C327801205C
:1025B000203A90400842F7D130782A280ED00222E3
:1025C000307801463039092916D804990A2359432D
:1025D000303940181443761C0490F1E7189802C86B
:1025E00004911890002904DA012040030443484272
:1025F000049002200443761C30782E2814D1042045
:1026000004437078761C2A2809D11898761C80C853
:10261000189009E00A214F43303FC719761C3078E3
:10262000014630390929F5D930786C2810D006DCFC
:102630004C281AD068280ED06A2817D104E07428D4
:1026400013D07A2812D110E00120400504430CE099
:102650000121090501E0032109050C43717881423C
:1026600003D1012000052418761C761C30781190C7
:1026700066280BD013DC58287DD009DC00287BD0DD
:102680004528F6D04628F4D047281AD1A5E118E00D
:10269000632835D0642870D0652812D19DE1702858
:1026A0006CD008DC6728F1D069287BD06E280DD06B
:1026B0006F2806D1BAE073282ED0752871D07828FB
:1026C00059D01A9A199990476D1C7EE16002400F0B
:1026D000022809D003280DD00428189801680DD0CD
:1026E0000D60001D189070E11898EA1701680D60E0
:1026F0004A60F6E7189801680D80F2E70D70F0E780
:1027000018986A4601781172001D189000205072C6
:1027100002A80090012005E0189802C81890002037
:102720000091C04361070DD5002101E00199491CCA
:102730000191B94212DA8142F8DB009A515C00291A
:10274000F4D10BE0002101E00199491C0191814283
:10275000FADB019A0099895C0029F5D10199049866
:102760001A9B471A21463846199A00F097FA0199A0
:10277000401945180BE04FE02CE113E04EE00098C3
:1027800000990078491C00911A9A1999904701986C
:10279000401E0190401CF2D1214638461A9B199ADE
:1027A00010E137E00A200021009001916002410F02
:1027B000022907D0189A01CA1892C2179446032911
:1027C00008D00AE01898C01DC108C90005C91891B1
:1027D000944607E000B2C2179446042902D140B2E1
:1027E000C1178C4600226146944506DA0A4600214C
:1027F000404291418C462D2102E0210504D52B2138
:102800006A461173012103E0E10701D02021F7E7B7
:10281000029155E00A200AE0102008E01020009004
:102820000021042004430191082703E0082000212F
:10283000019100906002410F022907D0189A01CA45
:10284000189200229446032908D008E01898C01D69
:10285000C108C90005C91891944603E080B2042953
:1028600000D1C0B200210291210729D51199702908
:1028700006D0009A1021019B4A401A4305D00EE071
:1028800040216A461173012108E06146014306D0E8
:1028900030216A4611731199517302210291009AF5
:1028A0000821019B4A401A430AD16146014301D1E4
:1028B000610705D530216A46117301217F1E0291FF
:1028C0001199582904D035A10E910DA90D910DE053
:1028D00037A1F9E76146019B009AFDF7CEFC0E9BFC
:1028E0008C469B5C0D9A521E0D92137061460143FB
:1028F000F0D10D9805A9081A20300190600703D582
:1029000001200004844300E001270198874201DD93
:10291000381A00E000200199009041180298091827
:102920000498401A0490E00306D421461A9B199A91
:10293000049800F0B3F94519002706E003A81A9A95
:10294000C05D199990476D1C7F1C02988742F5DB8A
:10295000E0030CD521461A9B199A049800F09EF9C1
:10296000451904E01A9A3020199990476D1C009976
:10297000481E00900029F5DC08E00D980D990078BC
:10298000491C0D911A9A199990476D1C0199481E7E
:1029900001900029F1DC63E1092801003031323374
:1029A000343536373839616263646566000000008B
:1029B0003031323334353637383941424344454675
:1029C0000000000000F05AF94519761C3078002804
:1029D00000D0E2E528461BB0F0BD600700D4062712
:1029E0001898C01DC108C90048680A680831C30F9B
:1029F000DB071891190001D09CA108E0210501D541
:102A00009BA104E0E10701D09AA100E09AA1430054
:102A100011985B08109165280CD006DC452809D078
:102A200046281DD0472841D141E0662818D06728A4
:102A30003CD13CE00021112F01DB112000E0781C8B
:102A40000191009008A911A8FFF7E8FC13990591DE
:102A50000021119A15927F1C12980197009150E065
:102A60000120C00703900120019008A9009711A838
:102A7000FFF7D4FC139A149905920022119B00923F
:102A800012981593059A0192002901D0104602E090
:102A9000791C40180190381A01D5019804E0404291
:102AA000401E0090781C0190C01B029043E0012F53
:102AB00000DA01270021112F01DD112000E0384646
:102AC0000191009008A911A8FFF7A8FC139905919E
:102AD000119A0021129815920091019721070CD4A8
:102AE0000599B94201DB019900E00191012904DD5A
:102AF000159A491E515C302906D0B84201DA011DF1
:102B000005DA0121029115E00199491EEDE700283F
:102B100005DC0099411800910199091A03E0019A16
:102B2000411C914200DD01910099401A401C029025
:102B30000120C0070390200706D402990198814222
:102B400002DB0020C043029000206946C87707AF2F
:102B5000012103980337C907884224D0022011902D
:102B60002B201290039800280CDA404203902D206D
:102B7000129007E00A210398FDF7BAFA30317F1E60
:102B8000039039701199481E11900029F2DC0398C6
:102B90000028EFD1791E1298087030782021084063
:102BA0004530BF1E387006A8C01BC01D039010988A
:102BB0000078002800D00120019941180298C01720
:102BC0000918039809180498401A401E0490E0035D
:102BD00006D421461A9B199A049800F05FF845190B
:102BE00010980078002803D01A9A199990476D1C04
:102BF000E00324D521461A9B199A049800F04EF858
:102C000045191CE00098002807DB009905988842C8
:102C100003DD1598405C199901E0199930201A9A42
:102C2000904700986D1C401C00900298401E029036
:102C3000002804D11A9A2E20199990476D1C0199E9
:102C4000481E01900029DDDC05E038781A9A7F1CC7
:102C5000199990476D1C0399481E03900029F4DCD4
:102C600021461A9B199A0498ACE600002D0000003A
:102C70002B0000002000000000000000F8B5044612
:102C800000251E461746880404D405E03946202056
:102C9000B0476D1C641EF9D52846F8BDFFB5044643
:102CA000002581B01E46C80301D5302700E020274B
:102CB000880404D505E038460399B0476D1C641EAE
:102CC000F9D5284605B0F0BD10B50420FEF716FD75
:102CD00001495520887510BD0000002010B50B4C2F
:102CE0000948606202210A48FEF7E4FE002809D084
:102CF000052020210007FEF7DDFE002801D000207E
:102D0000E07510BD0120FBE7204E00000000002010
:102D1000000800501CB5032405200094074B012235
:102D2000202100070194FEF7BDFD0094034B012212
:102D3000022103480194FEF7B5FD1CBDDD2C000007
:102D40000008005070B54049002208781346552805
:102D50006DD1CC783D48002C73D0012C0AD0022CC8
:102D600015D0032C21D0FF2C2DD0FE2C31D0FD2CE2
:102D70003CD048E04B78364A002B8B7802D0DB0001
:102D8000D25802E0DB009A18526805233BE0304A33
:102D90004B782832002B8B7802D0DB00D25802E02F
:102DA000DB009A18526806232DE0294A4B785832E6
:102DB000002B8B7802D0DB00D25802E0DB009A189F
:102DC000526809231FE0224A4B78383A04E0012375
:102DD00019E01F4A4B78303A002B8B7802D0DB0089
:102DE000D258F4E7DB009A185268F0E7184A4B789B
:102DF000A032002B8B7802D0DB00D25802E0DB003F
:102E00009A18526802238C8B641CA4B28C8394425F
:102E10000EDB00248C834A7801256A404A7010D06A
:102E20008A78521CD2B28A709A4204DBCC7070BD90
:102E30004978002905D001222021FEF78DFE70BDC2
:102E4000FFE70022F8E70000000000200004005027
:102E5000A84C000008B50020034600900122202164
:102E60000348FEF737FE03495520087008BD0000EF
:102E7000000400500000002005490A78552A05D1B9
:102E8000C870002088708883012048707047000057
:102E90000000002010B503780024C25C491E8B425C
:102EA00005D189B200F036F8002800D00124204670
:102EB00010BD00000C48416A002910D10B49097867
:102EC000002901D001290AD1C27C002A07D1022998
:102ED00005D0C17A002902D1C079002801D0002094
:102EE000704701207047000000000020C40000204F
:102EF0000149002048707047E0030020014900208C
:102F000088707047E0030020014900200870704776
:102F1000E003002070B515460723552200F022F883
:102F20000446014604A0FFF7FBF9AC4201D10120A1
:102F300070BD002070BD0000636D705F6372633808
:102F400020637263203D20307825780A000000005D
:102F500010B54418491E017089B2641E00F0E2F9F0
:102F6000207010BD30B5044610460FE02278504066
:102F70000022641C050603D54006000E584001E0FF
:102F80004006000E521CD2B2082AF3D30A46491E4C
:102F900089B2002AEAD130BD70B5314C206D01787C
:102FA00000291BD0E17D002918D10025057040784B
:102FB000012813D12B486062657600F097F901264D
:102FC00000281DD0FFF79AFFFFF792FFE572607AA5
:102FD000002804D0072000F0EBFEA67270BDFF2091
:102FE000FFF74AFF072000F0E3FE7D20C00000F05D
:102FF0001DFAFFF789FF6672002001F0B1F870BD7D
:1030000000F066F9002815D0FFF77EFF607A0028EF
:10301000F5D0FE20FFF730FF13481449C078800038
:10302000085801F061F9002001F09AF81048606238
:10303000E67170BD00F060F9002808D0FFF764FF6A
:103040006576A07A0028F4D06572A57270BD7D20E7
:103050000001FDF7D1FCFDF7DDFCFDF7C1FC70BD03
:1030600000000020204E000030010020804C0000B5
:10307000E093040070B5194C207D55280DD1E16B0B
:103080001748184D002909D0491EE16305D1602277
:10309000032101F08AFD6868A06370BD627D002A8B
:1030A000FBD0A16B0029F8D0491EA163F5D1521EB7
:1030B0001106090E61750CD0A968002904D01022F0
:1030C000032101F072FD01E06868A063A868E06375
:1030D00070BD1022032101F068FD70BD00000020CA
:1030E000000400405402002070B51F4D0446287DA6
:1030F0001E4E55280AD008218020FEF73FFD1022E1
:103100000321304601F051FD55202875632C00D96C
:1031100063240220687564220020121BE8635300B8
:103120001348D218A10082604160A9630A2C01D221
:1031300002200CE0142C01D2052008E01E2C01D244
:10314000072004E03C2C01D2082000E00A200821DE
:103150003446B162B821F16201F080F960220321A6
:10316000204601F022FD70BD000000200004004058
:103170005402002070B50020104903460C2242433F
:10318000144652189568002D14D05578002D11D191
:1031900055686D1C55609668761EB5420AD353601B
:1031A0000C5D002C00D19360054C01222568824003
:1031B0002A432260401C2028E0DB70BD6002002012
:1031C0005400002000B5012001F042F904490A68CA
:1031D000086848600020086001F03AF9104600BD18
:1031E0005400002010B50146012001F031F90C22F5
:1031F0004A43094B00201446D2189060506018557D
:1032000050700120884005490A681043086000207A
:1032100001F01EF910BD00006002002054000020E3
:1032200003498862CA6980231A42FBD070470000B4
:1032300000380140F8B51C4DA87D552801D000206C
:10324000F8BD1A4C01272760FEF7FEFAFEF7F4FAE4
:1032500006460020FEF74CFA02212160FCF7DEFF53
:103260003146FCF792FF0B21C943FCF7CBFF01214C
:10327000FCF7C8FFFCF7D9FF84B20D48844201D2A5
:103280002F7305E00B48844202D90020287368732D
:103290003046FCF7DEFF02460B4607A00094FFF71E
:1032A0003FF82046F8BD0000000000200024014047
:1032B000B80B0000E40C000068656C6C6F20776F41
:1032C000726C64202025662025750D0A0000000020
:1032D0000148407970470000E0030020012181404F
:1032E0000148406808407047540000200148807938
:1032F00070470000E003002001480079704700009B
:10330000E0030020064A00214B00D356834201DB34
:10331000C8B27047491C1729F6D316207047000021
:10332000F400002000B507235522FFF71BFE00BD67
:1033300000B5064B04485862FFF7BCFD002801D0D9
:103340000120587600BD0000204E00000000002043
:1033500010B5114C207E002801D0002010BD0020A7
:103360002064052040210007FEF7A4FB002801D1BE
:1033700001202064626C216C00208A4202D0072266
:10338000A26402E0A26C002A02D0521EA26400E0F5
:103390000846616410BD0000000000201CB502203A
:1033A0000321009001910520034B012240210007D9
:1033B000FEF778FA1CBD00003133000010B510494B
:1033C000887C552809D10A6B0E48002A0BD0521E62
:1033D0000A6303D08021FEF7B1FB10BD00228021DB
:1033E000FEF7BAFB10BDCA7C002AFBD04A6B7D23D6
:1033F000521CDB004A639A42F4D900224A63E9E78F
:10340000000000200004005008B500200346009092
:10341000012280210348FEF75DFB03495520887493
:1034200008BD0000000400500000002002498A7C12
:10343000552A00D1086370470000002003498A7CA8
:10344000552A02D100224A63C87470470000002048
:1034500010B51F48426801210A43426002234268B6
:103460001A40022AFBD11A4853044038C26B032485
:10347000A404A2431A43C263436BC20413434363CD
:1034800000BF00BF00BF134CE06807225202904308
:10349000E0601148036B020613430363436B9343DD
:1034A0004363A26802200243A260206908432061AE
:1034B000042001F011FA4B200002A06107480168C6
:1034C000090A09020160012005490005086010BDD4
:1034D00040100240007C00404018024014E400E02C
:1034E00000E100E01FB50220FEF70AFD01F08CF8B4
:1034F0002F200D22F6494002FEF758FA0D21F4481C
:10350000FFF7C8FC002804D10D22F249F048FCF76F
:1035100005FEFFF79FFC00F039FCFFF775FFFFF792
:10352000D3FBED4801F07CF8E121052307220903D4
:10353000EA48FEF79BFDFFF7EDFBFFF72FFF0520A5
:1035400040210007FEF7B6FAE54D002801D1012021
:10355000E872E449002000F025FD7D26F6000028F1
:1035600001D0FE2003E03046FFF760FFFF20FFF7A9
:1035700083FCD74CE01DFCF7F5FD411C02D0C006D2
:10358000C00EA070142000F0EFFE022000F070FECC
:10359000A0786179CF4F4843D349183F4843E17839
:1035A00089007958401800F09FFE452000F0D0FEB9
:1035B000002000F0D5FD0023CC4A1946CC48FEF788
:1035C00003FDFFF745FF00220A230121104600F00A
:1035D000E7FFFF230121F5330022084600F0E0FF5A
:1035E0003346002201210E2000F0DAFFC1A0FEF7D1
:1035F00097FEE178C2A0FEF793FEA178C4A0FEF783
:103600008FFEE01DFCF7AEFD0146C4A0FEF788FE6C
:10361000E17AC7A0FEF784FE052040210007FEF7EF
:1036200049FAAB4E01461036304616301536039037
:1036300000291AD1C248686201228021C148FEF7E0
:103640008BFAE078A84A800039586079504308180E
:1036500000F04AFEE078A44A80003958607950436F
:103660000918002000F01CFEFEE7FFF7ABFD00206C
:10367000FFF734FE002808D0FFF76AFEC0B2E876F4
:10368000FDF7CEF92865FFF787FC0120FFF726FE3E
:103690000E20FFF723FE0F20FFF720FE0A20FFF782
:1036A0001DFE002876D08A481030017D3046FFF795
:1036B000F1FB00286FD07078C106C90EA2A0FEF7FA
:1036C0002FFE039F78783978000208438005C10EE9
:1036D000A5A0FEF725FEB0780007810FACA0FEF78D
:1036E0001FFEE97DB2A0FEF71BFE697ABAA0FEF7C5
:1036F00017FE297BC2A0FEF713FE687AE97D2A7BBC
:10370000884390437ED07878397800020843820558
:10371000A778D00EB84207D1B078E17A0007800FC1
:10372000814208D0032806D07078C006C00E102849
:1037300031D1D00EFCD17D200001686200202871BB
:103740007178C906C90E10390B00FEF710FE060489
:10375000B47AC0BFBE24F078B17800020843317952
:103760000027090408430002000BE11DFCF704FDDB
:10377000C006C00EA070B0780D210007800FE07267
:103780005348FFF7E5FB0D2251492F20FEF718F9AA
:10379000014601E002E2FCE1A3A0FEF7C1FDB07822
:1037A0000007800F022802D1C82000F039FF6946C7
:1037B0004878400940011030487088784978000204
:1037C00008431F214901884369464870000A8870F0
:1037D000C0B2F3210840E17A8907090F084369461E
:1037E000887048880979B378090408439449327984
:1037F0000840F17812040902194311430902090B28
:10380000090100E0C2E1084369464880000C0871E4
:10381000FFF710FD01A90131FCF7AEFC014682A0C3
:10382000FEF77EFD0A216846FFF792FB0A216846F3
:1038300000F0CAFDFE20FFF71FFBEF710120287288
:10384000A7E1701DFCF78EFCC0B2FFF74DFC694686
:10385000487840094001163048708878497800025D
:1038600008431F2149018843A178C906890D0843EF
:1038700069464870000A8870C0B2F3210840E17AB6
:103880008907090F08436946887048880979B37821
:10389000090408436A4932790840F17812040902A0
:1038A000194311430902090B09010843694648807D
:1038B000000C0871C6E011206871701DFCF752FC05
:1038C000C0B2A87100F074FAD7E015E10AE1CCE0CB
:1038D00030010020984C0000DC0500000038014059
:1038E00000000020B544000010270000593C0000F3
:1038F0001C250000706F776572206F6E000000005D
:103900006672657142616E643A25640A00000000C7
:103910006368616E6E656C3A25640A007461726753
:103920006574496D65693A253038580A0000000011
:10393000646F67414273656C6563743A25640A007D
:1039400040771B00000400504556454E545F5246D8
:103950005F4745545F5041434B455420636D643A83
:10396000253032580A0000004556454E545F5246F5
:103970005F4745545F5041434B455420696E666F25
:10398000722E72664368616E6E656C3A25640A0039
:103990004556454E545F52465F4745545F5041433C
:1039A0004B455420747970653A25640A0000000084
:1039B0004556454E545F52465F4745545F5041431C
:1039C0004B455420626174436867537461466C616F
:1039D000673A25640A0000004556454E545F52463A
:1039E0005F4745545F5041434B4554206B657950C8
:1039F0006F7765724F6E466C61673A25640A000006
:103A00004556454E545F52465F4745545F504143CB
:103A10004B4554206261744C6F77566C74466C61F0
:103A2000673A25640A000000434D445F4445564907
:103A300043455F50414952202025640A00000000A0
:103A40000F0000FFFFF7F6FB01A90131FCF794FB23
:103A500001466A48FEF764FC0A216846FFF778FAD7
:103A60000A21684600F0B0FC93E0701DFCF77AFB79
:103A7000002800D00120FFF7E1FC684640784109AA
:103A80004901684616314170817840780902014346
:103A90001F2040018143A078C006800D0143684685
:103AA0004170090A8170C9B2F3200140E07A8007B1
:103AB000000F01436846817041880079B3780004A3
:103AC00001434F4832790140F07812040002184354
:103AD00010430002000B0001014368464180090CBD
:103AE0000171AFE714206871701DFCF73BFBC0B299
:103AF000A871FFF7C1F9C0E7701DFCF733FB0007A1
:103B000000D00120A873002801D0B42001E0E120FA
:103B10008000A8626846407841094901684615312D
:103B2000417081784078090201431F2040018143A0
:103B3000F806800D014368464170090A8170C9B2D8
:103B4000F3200140E07A8007000F0143684681704E
:103B500041880079B3780004014329483279014053
:103B6000F07812040002184310430002000B000119
:103B7000014368464180090C0171FFF75BFB01A915
:103B80000131FCF7F9FA01461EA063E723A0FEF716
:103B9000C7FBFF2115312648FCF7D9FA00F046FA99
:103BA000FFF788F9002800D15FE5224F3868400808
:103BB0004000386020A0FEF7B3FB0021012000F098
:103BC00095FE01F025F81FA0FEF7AAFB3868012139
:103BD00008433860687E002804D00020687600F032
:103BE000BFFA42E53C2000F0BBFA012000F052F998
:103BF0000021012000F07AFE37E50000283A00009D
:103C00000F0000FF434D445F52454241434B5F5319
:103C1000454E44202025640A000000006261744380
:103C20006867537461466C61673D25640A00000053
:103C300040010020002C01406C6F7720706F776589
:103C4000720D0A006C6F7720706F77657220776154
:103C50006B6575700D0A000070B5274CE08B401C39
:103C600080B2E083052829D10025E583FFF782FA99
:103C7000E06C2249401CE064884200D1E564606A3F
:103C8000002810D0401E6062E07918D000280AD0C9
:103C9000208C411C2184FF21F531884203D32584E7
:103CA0006420FFF7C3FB012000F070FB00F02EF84A
:103CB000FFF784FBFFF7DEF9FFF744F870BD00283B
:103CC0000DD00F48E57181784279C07851430D4A93
:103CD000800051430C4A1058081800F005FBE07CA6
:103CE0000028E0D1E07D002803D0002000F038FA61
:103CF000D9E73C20FAE7000000000020E9030000BB
:103D00003001002010270000804C000010B516493B
:103D1000C87B552824D1087C002821D0134A0001F3
:103D20008218487C8300D218803A536FCA6A521CAA
:103D3000CA62934214D80022401CC3B2CA620C4C1F
:103D40004B74032B05D30A744A740AA0FEF7E8FAF1
:103D500007E0012B05D060220121204600F025FF5D
:103D600010BD1022F8E7000000000020584D0000B0
:103D7000000400406D6F746F72576F726B4C657604
:103D8000656C203D20300D0A0000000010B50821B0
:103D90002020FDF7F3FE10220121034800F005FF6B
:103DA00002495520C87310BD0004004000000020E7
:103DB00070B5124CE17B55291ED12074002161742D
:103DC00001460FA0FEF7ACFA134D602201212846F0
:103DD00000F0EBFEE86A217C104A090189182039BD
:103DE000097C6422511A48431146FCF781F90246C6
:103DF0000121284600F0C0FE70BD00000000002038
:103E00006D6F746F72576F726B4C6576656C203D89
:103E10002025640D0A00000000040040584D0000F9
:103E2000FF2207490132CB6813409342FBD148611E
:103E3000C868402210404028FAD14869C0B2704793
:103E40000030014070B50D4CE06A002814D00C4DD4
:103E5000284600F019FC284600F094FC6D1E284608
:103E600000F012FC284600F08DFCFCF7CDFF01208D
:103E7000207004A0FEF754FA70BD0000C4000020BA
:103E8000030000066D79526164696F5F61626F7251
:103E9000740A000010B500F0C3FB10BD70B500F04F
:103EA000B7FE0526360708213046FDF703FE0F4C06
:103EB000024621780EA0FEF733FA2078042814D1A8
:103EC0000025257008213046FDF7F4FD00280CD0B0
:103ED0000BA06561FEF724FA0C4800F053FC0B4878
:103EE000401E00F05BFC0320207070BDC400002069
:103EF000636164203D2025643D2025640D0A000097
:103F00006770696F4361640A0000000003000006E7
:103F10000149012008727047C4000020F8B5012350
:103F20000546022219461846FDF712FF00221146E7
:103F30000420FDF78FFF0A20FDF7BEFE0F4E002480
:103F400001231A46022130460094FDF7C3FD0023E9
:103F50001A46042130460094FDF7BCFD05200023DD
:103F60000122082100070094FDF7B4FDFCF7AAFC2C
:103F700000F008F802480560F8BD00000004005099
:103F8000240100201CB50321012001910090034B66
:103F9000002204210248FDF785FC1CBD490F0000EA
:103FA000000400507CB50C461448FFF7B7FF03200F
:103FB000009001900520124B002208210007FDF718
:103FC00071FCFCF7CDFF002804D00EA0FEF7A8F985
:103FD00000207CBDFCF7C0FE0E4D6878FDF7D2F9DD
:103FE0000A2000F01DFB002C00D0AC62E520E86246
:103FF00009A0FEF795F901207CBD0000113F0000EB
:104000009D3E00002020524620496E697420466182
:10401000696C0000C40000206D79526164696F5FB3
:10402000696E6974204F4B0A00000000F0B5434DE3
:10403000FFB0E86A8AB000287DD0287A00287AD0BC
:1040400000262E7229783EA0FEF76AF92878022809
:1040500001D003286FD1FCF74FFF044601463CA076
:10406000FEF75EF945A8E107879016D0FDF786FABE
:104070000120FCF71FFE64086400FCF7FFFE2E70B1
:10408000AF6A002F09D0FF22093268468799FCF7F2
:1040900045F842A90EC90320B84720071CD5FCF7F4
:1040A00039FF40A9088247A80130FCF73AFF40A930
:1040B00008770820FCF7FEFD2E70F720AF6A044059
:1040C000002F09D0FF22093268468799FCF726F8AD
:1040D00042A90EC90020B847600712D50420FCF79A
:1040E000E9FD2E70FB20AF6A0440002F09D0FF22AB
:1040F000093268468799FCF711F842A90EC90220D7
:10410000B847A00712D50220FCF7D4FD2E70FD2081
:10411000AD6A0440002D09D0FF2209326846879914
:10412000FBF7FCFF42AE0ECE0120A847002C02D0C8
:104130002046FCF7BFFD7FB00AB0F0BDC4000020F0
:1041400072665F70726F636573733D25640A000069
:10415000495251466C61673D307825580A0000008D
:1041600070B52B4C0546E06A00284FD00020E06077
:1041700020616061274EA061304600F085FA30462C
:1041800000F000FB24A0FEF7CBF82078022802D034
:10419000032802D004E024A036E026A0FEF7C0F8F1
:1041A0002078042804D126A0FEF7BAF8FDF7CAF952
:1041B000FCF7AAFE002812D100210846FFF7F2FE04
:1041C000206A00F091F80220205600F0CDF8A27984
:1041D0006179207900F0A6F8012000F021FAFCF7BF
:1041E00093FE012801D1FCF753FE002D03D0A8B2A5
:1041F000FCF7F6FD01E0FCF7E4FD0648401E00F088
:10420000CDFA0320207015A0FEF78AF870BD0000DB
:10421000C400002003000006737461727420746F80
:104220002072780A000000004E4F57204953207436
:10423000780A00004E4F572049532072780A000038
:104240004E4F57204953204341442072782C20542C
:104250004F2053544F50204341440A005355434389
:1042600045535320454E5445522072780A000000B1
:1042700070B50949CA6A002A0DD048624100074E4C
:104280004518AC19A078FCF75FFF705DFCF742FFA2
:104290006078FDF7A7F870BDC40000208C4E0000C8
:1042A00070B5104C0646E06A002814D0052525702C
:1042B000452000F04DF8002E03D0012E0CD0022E28
:1042C00009D10220205600F04FF8206A00F00CF8C7
:1042D000FDF716F9257070BD0020FFF741FF0320A0
:1042E000207070BDC400002010B5064CE16A0029A2
:1042F00006D02062FCF786FF03A0216AFEF710F8C3
:1043000010BD0000C40000206D79526164696F5FC8
:104310007365744672657175656E63793D25750ABE
:104320000000000070B5054608480C46C16A002927
:104330000BD00571447182711046FCF705FF2046D1
:10434000FCF7E8FE2846FDF74DF870BDC4000020DC
:1043500010B50449CA6A002A02D0C870FDF750F8A7
:1043600010BD0000C400002010B50749CA6A002A29
:1043700009D08870FEF7C6FF03494000303140186D
:104380004078FDF751F810BDC400002070B50C4C0A
:104390007D21E069C900401C0025E061884200D908
:1043A000E561606900280AD0401E606107D10548B8
:1043B00000F0E8F9FDF7C6F82570FCF725FD70BDA3
:1043C000C40000200300000670B5194C0646E06AE0
:1043D0000D4600282BD0FCF797FD002812D10021B4
:1043E0000846FFF7DFFD206AFFF77EFF0220205618
:1043F000FFF7BAFFA27961792079FFF793FF0A20CE
:1044000000F00EF9FCF780FD012804D1FCF740FD17
:104410000A2000F005F9E9B23046FDF7E3F8054857
:1044200000F0BCF90220207003A0FDF779FF70BDF9
:10443000C4000020020000066D79526164696F5F5C
:104440007472616E736D697441727261790A0000F1
:10445000002800D0012080F31088704770B5044612
:10446000642800D96424094DE96A09A0FDF758FFC2
:10447000E86A6421091B48436421FBF739FE0246C0
:104480000321284600F078FB70BD000000040040C6
:104490007374645F74696D5F6765745F6175746F71
:1044A00072656C6F61642854494D33293D25640A57
:1044B000000000000FB430B50446014687B028A0C4
:1044C000FDF72EFF294D002C23D0012C45D0022CC6
:1044D00017D0032C18D1287A002812D00020244CA1
:1044E0002872A0786179244A484322494843E178F8
:1044F000890051584018FFF7F7FEA1781FA0FDF77B
:104500000FFF0020FFF72CFE07B030BC08BC04B042
:10451000184710A8837A427A017AC07903AC0FC495
:1045200010A88279417900796B4607C310A8C37837
:10453000827841781848FDF7F3FE0D48FF221532C6
:104540000BA91030FBF7EAFD0020FFF709FE0A2057
:10455000FEF748FE11486862D6E7FFF773FCD3E721
:104560007374617475733A25640D0A0000000020AD
:104570003001002010270000804C0000706169723B
:104580002073756363657373206368616E6E656C19
:104590003D25640D0A000000E0510000204E00009F
:1045A000F0B504460120FFF753FF20460C250A4EC4
:1045B00068438519AB6000276F6031546F70521EDD
:1045C000134205D1054901200A68A0401043086044
:1045D0000020FFF73DFFF0BD6002002054000020E6
:1045E000014610B50348044A00885043FBF780FD9C
:1045F00010BD0000C003FF1FE40C00000149096961
:104600000840704700240140044801690422114316
:1046100001610169012211430161704700E000E07E
:1046200070B57D250446ED0002E0284600F004F850
:10463000641EFAD270BD000010B504460B480A494A
:104640000068FBF755FD012160430906884200D947
:1046500008460749401E4861002088610869000C2F
:10466000C007FBD010BD000040420F00C00000207A
:1046700000E000E0C106C90E0120884001498860C1
:10468000704700000018024004494A68C306DB0E68
:104690000120984082434A607047000000180240A1
:1046A00003498968C206D20E012090400840704735
:1046B00000180240F0B50268314F5101890F36D021
:1046C000017A8C072E49A40F40394D68D606012285
:1046D000F60E1346B3409D434D6003780D68DB062C
:1046E000DB0E16469E40B5430D60E30707D0037806
:1046F0000D68DB06DB0E16469E4035430D60A307B2
:1047000006D503784C68DB06DB0E9A4014434C60F8
:1047100001684A01920F032A09D1C2683B69CC069D
:10472000640E0325A540AB43A24013433B610179CE
:1047300002788C073D6BA40F3946D6060122F60E8F
:104740001346B3409D433D6303787D6BDB06DB0E70
:1047500016469E40B5437D63E30707D003780D6B93
:10476000DB06DB0E16469E4035430D63A30706D5D8
:1047700000784B6BC006C00E824013434B63F0BD04
:104780004018024004490A68C306DB0E0120984025
:1047900082430A60704700000018024004490A681A
:1047A000C306DB0E0120984002430A6070470000F8
:1047B0000018024070B50D46002400F021F8601E7C
:1047C000012208491204286008691042FCD10869D6
:1047D000C00600D5012404480861002000F010F84C
:1047E000204670BD002002401000000103490A6805
:1047F0005208520002430A60704700000020024045
:1048000003494A6906239A4302434A6170470000FC
:104810000020024070B506460D4600240220FFF736
:10482000EFFF012109480904356002690A42FCD101
:104830000169C90602D43168A94200D001240449A3
:1048400001610020FFF7DCFF204670BD0020024020
:104850001000000110B5006849434A008A18104052
:10486000FBF746FC10BDF0B5002323E022460124EF
:104870009C4022401DD04F68066814465443650092
:104880006519AE4367433E4306608F68C668AE4312
:1048900025467D432E43C6604D68022D09D10E6921
:1048A000056A544354432201121B95437443254324
:1048B00005625B1C0A681446DA40D7D14A68012AAF
:1048C00001D0022A06D1CB684168224691435A435F
:1048D00011434160F0BD000003490A6906239A4371
:1048E00002430A6170470000007C004010B50F4A87
:1048F0000124536B24072343536300BF00BF00BF51
:104900000B4A13685B085B000343136009480369A3
:10491000042213430361002906D040BF20BF20BFFB
:1049200001699143016110BD30BFF9E700100240F9
:104930000070004000ED00E000B500F01FF80349F2
:1049400089684905490FC84000BD000000100240B9
:1049500000B5FFF7F1FF044989684904490F0329AD
:1049600001D3C91EC84000BD001002400248806843
:104970003821084070470000001002400948816853
:1049800038200140082905D0102905D0182905D064
:104990000548704705487047054870477D2000026C
:1049A000704700000010024000127A000024F4005A
:1049B000006CDC020349CA6A0243CA6200BF00BF3E
:1049C00000BF7047001002400349CA6A0243CA622E
:1049D00000BF00BF00BF7047001002400349CA6A11
:1049E0000243CA6200BF00BF00BF70470010024010
:1049F0000349CA6A0243CA6200BF00BF00BF7047D2
:104A0000001002400349CA6A0243CA6200BF00BFE5
:104A100000BF7047001002400349CA6A0243CA62DD
:104A200000BF00BF00BF70470010024003498A6802
:104A3000D208D20002438A60704700000010024092
:104A400010B54268816803690A43C16819430A4383
:104A500006490B68FF243F34A3431A430A600A68DF
:104A6000402300689A4302430A6010BD00300140B1
:104A7000124A10B590420FD1026860239A43026037
:104A8000CB684A681A43036837242401A3431A43B6
:104A900002600A7C026309E0094A904206D102687A
:104AA00003231B029A43CB681A4302608A68C262DE
:104AB000096881620121416110BD0000002C0140A4
:104AC00000040040FCB553009C46046A9300052591
:104AD0009D40AC4304620D680195D50700D00825C0
:104AE0009607F60F0096B6008419A6697327AF40A3
:104AF000BE43019FAF403E43A661046A03259D402B
:104B0000AC434E680D6935439D402C430462CC682C
:104B100005682D0406D41A18556B2D0C2D04254359
:104B200055630CE0009EF5007600921B920012186F
:104B3000566BFF27AF40BE43AC40264356630D4A39
:104B4000904216D14268032465462402AC40A24339
:104B5000CD698C692C436546AC4022434260026AB1
:104B60000C249C40A2434C6989680C439C4022431E
:104B70000262FCBD002C014010B503681B0405D483
:104B800089000818416B090C09040BE08B07DC0F46
:104B9000E3006400091B89000818416BFF249C4056
:104BA000A1439A401143416310BD10B5CB0700D01B
:104BB00008238907C90F89004018816973249C4024
:104BC000A1439A401143816110BD000070B50546B4
:104BD0000C46886809682A68084321690B4B1A400B
:104BE000114308432860E16868680122520390433A
:104BF00008436860FFF7ACFE6168002904D04A08EA
:104C00001018FBF775FAE86070BD0000F3E9FFFFCC
:104C1000134901200A68824302430A60114801686F
:104C2000821511430160011502680A408A42FBD1D6
:104C300082680221D208D2000A4382603822816849
:104C400011401029FBD18168072212029143816033
:104C500081681201914381600449034808607047EC
:104C60000020024000100240006CDC02C000002066
:104C7000E80300006400000032000000640000004F
:104C8000C0ACEF11C0BA1619C041AA1C401432338F
:104C9000003EFF3580264B0900000101166445FFE8
:104CA000FFFFFF0000000000320000006400000071
:104CB00032000000640000003200000064000000C8
:104CC00032000000640000003200000064000000B8
:104CD000C800000064000000C8000000640000007C
:104CE000C800000064000000C8000000640000006C
:104CF0003200000064000000320000006400000088
:104D000032000000320000003200000032000000DB
:104D100032000000320000003200000032000000CB
:104D200032000000320000003200000032000000BB
:104D300032000000320000003200000032000000AB
:104D4000320000003200000064000000C8000000D3
:104D500064000000C800000028000000900100006E
:104D600000000000000000003C000000A401000062
:104D7000000000000000000050000000B80100002A
:104D8000000000000000000050000000CC01000006
:104D900000000000000000005A000000E0010000D8
:104DA000000000000000000064000000F4010000AA
:104DB000000000000000000064000000E8030000A4
:104DC000000000000000000064000000640000001B
:104DD0000000000000000000020008001000400079
:104DE00080000800400001000100080010002000C1
:104DF00040008000010010002000000001000200BF
:104E000002002000010002000400040080000200F3
:104E10000100010008001000020002000400200050
:104E200080008000080000004000000080000000BA
:104E30000100000010000000400000000100000020
:104E400004000000100000008000000020000000AE
:104E50008000000010000000200000004000000062
:104E600008000000400000000400000000000006F0
:104E70000100000602000006030000060400000610
:104E8000050000060600000607000006060C0206E4
:104E900009040709030708020808020908010907AD
:104EA00001090701020406080C10040401010003B3
:104EB000010103F03005018105A18105F0810701A1
:104EC000810501800531800701800721800B118059
:104ED0000B21800B41800B61800B91800BB1800D09
:104EE000B1800FB180115080153020155070000036
:104EF0000000031B000476000601000B04001304ED
:104F0000001120001210001F0700200700240300DA
:104F1000460300250000210700220700152100316B
:104F2000D000366600376B0038CC003909003CB43D
:104F3000003E4200406A0041060042AA0048770055
:104F40004977004A77004B05004F040050D2005EBD
:104F50008001031B010476010B08010F0A011900EF
:104F6000012FD00143DA02031B020476022CC00297
:104F70002D27022E09022F0002301003031B030409
:104F800076030A0E030BCF030C19030D98031216B8
:104F90000313140316F4031701031FD990BF3E082F
:104FA000D00A8B082A0CC000D00A8B081056D708EC
:104FB0003A0CC0001056D708C01C3D094A0CC0006E
:104FC000C01C3D0940AA98095A0CC00040AA980983
:104FD000007A030A6A0CC000007A030A0095BA0A34
:104FE0007A0CC000E0325E0CC0A3D00C2A08B000DE
:104FF000C0A3D00CA014430D3A08B000A014430D78
:1050000020ABDB0D4A08B00020ABDB0DA041740ED5
:105010005A08B000A041740E20D80C0F6A08B000E6
:1050200020D80C0F80DF17107A08B000A09BD61094
:10503000C0451B112A06A000C0451B1140DCB3115E
:105040003A06A00040DCB31180397A124A06A0006B
:1050500080397A12C09640135A06A000C0964013B9
:10506000403616146A06A00040361614002A75153C
:105070007A06A00000965118C065BC181A06900068
:10508000C065BC188047A1192A0690008047A11965
:105090004029861A3A0690004029861A4056B71BC6
:1050A0004A0690004056B71B4083E81C5A06900001
:1050B0004083E81C40B0191E6A06900040B0191EDB
:1050C00000BF2F207A069000809E473080CB783139
:1050D0001A02800080CB7831008F42332A02800090
:1050E000008F423380520C353A02800080520C35DA
:1050F00080AC6E374A02800080AC6E378006D139B2
:105100005A0280008006D1398060333C6A028000F8
:105110008060333C007E5F407A0280000600F80623
:105120000600F8060600F8060600F80614C0F91492
:1051300022D4F92230D8F9303EDEF93E0EFF804FFE
:10514000128038010A0000000C0000000F0000006F
:10515000130000001A0000002000000028000000DA
:105160003300000041000000510000006600000014
:1051700080000000A2000000CC000000010100003F
:1051800044010000970100000102000085020000B8
:105190002D03000000040000080500005706000071
:1051A000FB0700000C0A0000A50C0000EE0F000039
:1051B0000B1400003E190000C21F00000028000070
:1051C00024F4000048E8010090D0030020A107006B
:1051D00000007A420000FA4200007A430000FA43DD
:1051E0007265636569766520646174613A25303261
:1051F000582025303258202530325820253032585A
:105200002025303258202530325820253032582081
:1052100025303258202530325820253032580D0A9A
:105220000000000044520000000000203001000097
:105230003208000088520000300100209006000073
:105240000C24000071021E0233204E033884030236
:1052500060010332127A702FE601EF02FB03FD04B6
:10526000FE05FF06020704080509070A080B090CDA
:105270000A0D0B0E0C0F0D100E110F12101311143E
:0852800012151316141682FF2B
:04000005000000C136
:00000001FF
